:100000000C9420060C9458060C9458060C94580630
:100010000C9458060C9458060C9458060C945806E8
:100020000C9458060C9458060C94A6270C94782827
:100030000C94DC210C9458060C9458060C94580629
:100040000C9458060C9458060C9458060C945806B8
:100050000C9458060C9464220C9458060C94580680
:100060000C9458060C9458060C9458060C94580698
:100070000C9458060C9458060C9458060C94580688
:100080000C9458060C9458060C9458060C94580678
:100090000C9458060C9458060C9458060C94580668
:1000A0000C9458060C9458060C945806260A260AF6
:1000B000520A520ABA0AD80AF00BF00BE30A7C0B78
:1000C0008D0B8D0BE5280C29042A0C29042A5829AC
:1000D0007B29042AD229E129290035001E001F00AE
:1000E00020002100220001522300240025002600C8
:1000F00027002D002E002B0014001A000800150008
:1001000017002F00000030001C0018000C00120027
:1001100013002A00035104001600070009000A001A
:100120004A0000004B000B000D000E000F003300D2
:100130002800E1001D001B000600190005004D000D
:100140004C004E0011001000360037003800E5006A
:100150000251E000E300E2002A0000000000280055
:1001600000002C42E7005000510052004F000100F7
:100170000100010001000100010001000052010026
:10018000010067005400550001000100010001005A
:100190000100ED000100010001000000010001006C
:1001A0005F0060006100560001000100F200EF00F6
:1001B000EE00F000010001000000010001005C0001
:1001C0005D005E005700010001000100FD00FE001F
:1001D000FF000100010001000100010059005A0068
:1001E0005B00580001000100010001000100010056
:1001F00000000000620000000100010063005800E0
:1002000001000100005C01003A003B003C003D00A1
:100210003E0001003F004000410042004300440016
:10022000450035001E001F002000210022000100B3
:1002300000000100230024002500260027004C00B8
:1002400001001E021F02200221022202AA00000059
:10025000A900230224022502260227020100010030
:100260002E022D002E002F023002AC00AE00AB009B
:100270002F00300033003302310001000100010083
:1002800001000100010000000000010000004C001E
:100290000100010001000100010001000100010056
:1002A0000100010001000100010001000100010046
:1002B0000100010001000100010001000100010036
:1002C0000100010001000000010001005004520083
:1002D0004F040100010001000100E000E200E10024
:1002E00001000100000001002A00500051004F00F1
:1002F0004C00010001001D081B0806081908010038
:100300000100010001000100500801004F08010038
:1003100001000100010001000100010000000000D7
:1003200001000000010001000100010001000100C6
:1003300044454255473A2064697361626C65642E96
:100340000A0044454255473A20656E61626C656417
:100350002E0A000A0025303258006C65645F746113
:10036000736B3A20004F6E6573686F743A20616357
:10037000746976653A2025640A000A002530313612
:1003800062003A200025303258000A722F63203074
:100390003132333435363738394142434445460AE1
:1003A00000290A002575002F002575005D2800250D
:1003B00064002000256400200025640020002564DE
:1003C000007C0025303258006D6F7573656B657960
:1003D000205B62746E7C782079207620685D2872BC
:1003E00065702F61636C293A205B00313A096465BE
:1003F0006C6179282A31306D73293A2025750A32CB
:100400003A09696E74657276616C286D73293A20B9
:1004100025750A333A096D61785F73706565643AD2
:100420002025750A343A0974696D655F746F5F6DD4
:1004300061783A2025750A353A09776865656C5FF9
:100440006D61785F73706565643A2025750A363A88
:1004500009776865656C5F74696D655F746F5F6D62
:1004600061783A2025750A00703A097072696E74D5
:100470002076616C7565730A643A0973657420644B
:10048000656661756C74730A75703A092B310A647C
:100490006E3A092D310A6C743A092B31300A7274A4
:1004A0003A092D31300A4553432F713A0971756964
:1004B000740A0A7370656564203D2064656C74611C
:1004C000202A206D61785F7370656564202A20287A
:1004D000726570656174202F2074696D655F746F3B
:1004E0005F6D6178290A77686572652064656C7450
:1004F000613A20637572736F723D25642C207768B2
:1005000065656C3D25640A53656520687474703AAE
:100510002F2F656E2E77696B6970656469612E6F28
:1005200072672F77696B692F4D6F7573655F6B65A8
:1005300079730A004D3E20004D25753A25733E2003
:10054000003F0A003D2025750A003F0A00646566E9
:1005500061756C74730A0025750A003F0A000A0968
:100560002D2056616C756573202D0A00710A000AF2
:10057000092D204D6F7573656B6579202D0A003F3D
:1005800000433E20004C25640A000A092D205374C4
:1005900061747573202D0A686F73745F6B6579627F
:1005A0006F6172645F6C65647328293A202530326C
:1005B000580A6B6579626F6172645F70726F746FF5
:1005C000636F6C3A20253032580A6B6579626F612F
:1005D00072645F69646C653A20253032580A746928
:1005E0006D65725F72656164333228293A20253067
:1005F000386C580A000A092D2056657273696F6EAF
:10060000202D0A5649443A20307837323732285262
:100610006F6D696E526F6E696E2043616E64794BC7
:1006200065797329205049443A2030784630334266
:10063000284B6174616E61363020726576322920F4
:100640005645523A203078303030310A4255494CC4
:10065000443A202028466562203238203230323237
:10066000290A4F5054494F4E533A204C5546412089
:100670004D4F5553454B45592045585452414B45D4
:100680005920434F4E534F4C4520434F4D4D414E03
:100690004420343039360A4743433A20352E342E2D
:1006A00030204156522D4C4942433A20322E302EB2
:1006B00030204156525F415243483A2061767235AC
:1006C0000A000A092D20436F6E736F6C65202D0A96
:1006D0004553432F713A09717569740A6D3A096D72
:1006E0006F7573656B65790A000A092D204D616786
:1006F0006963202D0A443A094465627567204D6597
:10070000737361676520546F67676C650A583A09AF
:100710004D6174726978204465627567204D6F641D
:100720006520546F67676C65202D2053686F7720B4
:100730006B65797072657373657320696E206D6186
:100740007472697820677269640A4B3A094B65795B
:10075000626F61726420446562756720546F6767D9
:100760006C65202D2053686F77206B6579707265FA
:100770007373207265706F72740A4D3A0944656232
:100780007567204D6F75736520546F67676C650AD8
:10079000563A0956657273696F6E0A533A09537473
:1007A000617475730A433A094163746976617465CB
:1007B00020436F6E736F6C65204D6F64650A463120
:1007C0002D4631303A0953776974636820746F207D
:1007D0004C6179657220302D392028463130203D1A
:1007E000204C30290A302D393A09537769746368EF
:1007F00020746F204C6179657220302D390A475280
:100800004156453A0953776974636820746F204CE8
:100810006179657220302028616C7465726E617434
:1008200065290A423A094A756D7020746F20426F3B
:100830006F746C6F616465720A4553433A094A7577
:100840006D7020746F20426F6F746C6F616465729D
:100850002028616C7465726E617465290A453A09D5
:100860005072696E7420454550524F4D2053657447
:1008700074696E67730A4253504143453A09436CA9
:1008800065617220454550524F4D0A006B65796D88
:1008900061705F636F6E6669672E7261773A2025BB
:1008A0003032580A2E737761705F636F6E74726FA7
:1008B0006C5F636170736C6F636B3A2025750A2EF1
:1008C000636170736C6F636B5F746F5F636F6E7483
:1008D000726F6C3A2025750A2E737761705F6C63B6
:1008E000746C5F6C6775693A2025750A2E737761A1
:1008F000705F7263746C5F726775693A2025750A60
:100900002E737761705F6C616C745F6C6775693AA8
:100910002025750A2E737761705F72616C745F7247
:100920006775693A2025750A2E6E6F5F6775693A9B
:100930002025750A2E737761705F67726176655F37
:100940006573633A2025750A2E737761705F626163
:10095000636B736C6173685F6261636B7370616317
:10096000653A2025750A2E6E6B726F3A2025750A3E
:100970000064656275675F636F6E6669672E72619A
:10098000773A20253032580A2E656E61626C653ADE
:100990002025750A2E6D61747269783A2025750AD2
:1009A0002E6B6579626F6172643A2025750A2E6D2F
:1009B0006F7573653A2025750A006565636F6E660D
:1009C00069673A0A64656661756C745F6C61796524
:1009D000723A2025750A003F000A6D6F7573653AFB
:1009E000206F66660A000A6D6F7573653A206F6E38
:1009F0000A000A6B6579626F6172643A206F6666FD
:100A00000A000A6B6579626F6172643A206F6E0A40
:100A1000000A6D61747269783A206F66660A000A8E
:100A20006D61747269783A206F6E0A000A646562BB
:100A300075673A206F66660A000A64656275673AF0
:100A4000206F6E0A000A0A4A756D70696E6720741D
:100A50006F20626F6F746C6F616465722E2E2E2032
:100A600000433E2000436C656172696E6720454516
:100A700050524F4D0A000A002530325820006B6555
:100A800079626F6172645F7265706F72743A200090
:100A90005B735D005B575D005B535D005B525D0007
:100AA0005B445D005B435D001C034B006100740010
:100AB00061006E00610036003000200072006500A9
:100AC0007600320000002A0352006F006D006900BA
:100AD0006E0052006F006E0069006E00200043003F
:100AE00061006E00640079004B00650079007300BE
:100AF00000000403090409025B00030100A0FA09D5
:100B0000040000010301010009211101000122403C
:100B1000000705810308000109040100010300002A
:100B200000092111010001227B000705820320003A
:100B30000109040200020300000009211101000163
:100B4000222200070583032000010705030320007C
:100B500001120100020000000872723BF001000166
:100B60000200010631FF0974A1010975150026FF75
:100B7000009520750881020976150026FF00952052
:100B800075089102C005010902A10185020901A1B0
:100B9000000509190129081500250195087501812D
:100BA000020501093009311581257F9502750881FB
:100BB0000609381581257F950175088106050C0AFF
:100BC00038021581257F950175088106C0C0050191
:100BD0000980A101850319012AB700150126B70074
:100BE000950175108100C0050C0901A1018504194A
:100BF000012AA002150126A002950175108100C0EE
:100C000005010906A101050719E029E715002501DD
:100C10009508750181029501750881010507190084
:100C200029FF150026FF00950675088100050819A3
:100C3000012905950575019102950175039101C082
:100C400011241FBECFEFDAE0DEBFCDBF04B603FE36
:100C500018C08091F2029091F302A091F402B09139
:100C6000F5028730904BA740B04B59F41092F20236
:100C70001092F3021092F4021092F502E0E0F8E311
:100C8000099511E0A0E0B1E0E4E8F5E502C00590C7
:100C90000D92AC3FB107D9F722E0ACEFB1E001C053
:100CA0001D92A23FB207E1F70E9433180C94C02AAC
:100CB0000C940000FF93EF93E091FC01F091FD0193
:100CC000309709F00995EF91FF910895FC01859106
:100CD000803011F0EFDFFBCF0895FF27E0E230E234
:100CE00047FF0CC0419597FF09C0EDE260957095F4
:100CF00080959095611D711D811D911D27FF02C07A
:100D0000219530E350E2AA27660F771F881F991FAD
:100D1000AA1FA41710F0A41B63955A95A9F7AA302F
:100D200008F0A95FA05DAF93F3956115710581058A
:100D3000910541F7ED3211F4EF93F395F21718F4A2
:100D40003F93F395FBCF8F91B5DFFA95E1F70895C7
:100D5000E991F9918591803021F0853219F0AADF6F
:100D6000F9CF089520E0E89455915532C1F35033FE
:100D700011F4689455915A3348F4505390F3220F6C
:100D8000022E220F220F200D250FF4CF0EF42195F5
:100D900089919991533619F3533729F1533559F104
:100DA000BC0188279927E8945C3621F489919991B0
:100DB00068945591543639F446EF7EF077FF0DC0B4
:100DC0008FEF9FEF0AC055374AE039F0583540E1C0
:100DD00021F0523642E009F00895FF93EF937DDF52
:100DE000EF91FF91B7CFFF93EF93FC01819180309A
:100DF000B9F360DFFBCFFF93EF9368DFF1CFDF93B1
:100E0000CF93CDB7DEB72596A3DFCF91DF910895BD
:100E100081E0089581E008950C940A0708950C94E8
:100E20000E071F93CF93DF9300D000D01F92CDB752
:100E3000DEB749835A836B833091FF0189819A81A0
:100E4000311114C0662359F0222349F00E942D0E5F
:100E5000182F682F89819A810E94D60D03C00E94A5
:100E6000010E182F69817A81812F04C00E942D0EF6
:100E700069817A810F900F900F900F900F90DF9102
:100E8000CF911F910C947115FC01262F4081518147
:100E90006281738184810C94110781E00895CF935E
:100EA000DF93EC0160E00E944407BE01DF91CF9127
:100EB0000C940F070C94E4160C94E01608950E940D
:100EC000800C0E945E072FEF84E39CE0215080405D
:100ED0009040E1F700C000000C948A220F931F930A
:100EE000CF93DF938C0161E00E944407EC01B801CD
:100EF0000E940C07882309F45BC0B801CE010E9450
:100F00006920882309F454C0B801CE010E944B1B0C
:100F1000882309F44DC0B801CE010E94C51F882363
:100F200009F446C0F80182818823D9F1CF3D8CE5D0
:100F3000D80779F140F4C115FCE5DF0791F0C13025
:100F4000DC4591F02EC0CC35EDE5DE0741F1CD3525
:100F5000FDE5DF0709F1CB35DD4519F50E94C41227
:100F600020C00E945F0724C080919802C82FC095BE
:100F7000C170C0FB80F980939802CC2329F082E4F1
:100F800093E00E94660614C080E393E00E94660628
:100F900010C00E9472130CC00E94BB1202C00E94BB
:100FA000C712C801DF91CF911F910F910C940807D0
:100FB000C0E08C2FDF91CF911F910F9108950E9477
:100FC000BE210C941D080E9420080C94C421829517
:100FD000982F937344E0949F900111248C7C869504
:100FE0008695282B822F8575880F2A7A2695822B45
:100FF0000895CF93DF93D92F0E94E707C82F8D2F35
:101000000E94E7072C2F30E0322F2227A901482B1E
:10101000CA01DF91CF91089508950C940C0881E0E6
:1010200008950C940F080895CF93C82F0E940D08BF
:101030008C2F0E941108CF91089580E00C94140821
:101040000E94C5200C941408CF930E94C520C82F7D
:101050008091FE01C81741F1C093FE018091980272
:1010600082FF1EC080FF04C08AE593E00E946606EE
:101070008091980280FF0CC01F92CF9385E593E08A
:101080009F938F930E94FF060F900F900F900F90E9
:101090008091980280FF04C083E593E00E94660679
:1010A0008C2FCF910C941408CF910895CF93DF9398
:1010B000CDB7DEB72B970FB6F894DEBF0FBECDBF0E
:1010C0004F83588769877A878B8761110E94F31154
:1010D0009E012F5F3F4F86E0F90111928A95E9F753
:1010E00085E0FE013796D90101900D928A95E1F7CE
:1010F00089819A814C815D81452B31F09F3F31F48C
:1011000091E08F3F19F403C091E001C090E090FF9F
:1011100009C049815A816B817C818D819E810E94A9
:10112000141105C0C9010E944D078111F2CF2B9601
:101130000FB6F894DEBF0FBECDBFDF91CF910895FB
:10114000FC01808191810E946F0E0895CF938823C6
:1011500009F4A9C0C82F8238C1F40E94C52081FDBE
:10116000A2C069E380910201909103010E9496213F
:101170000E9415122FEF81EE94E0215080409040A4
:10118000E1F700C0000069E319C0833801F50E944F
:10119000C52080FD88C063E5809102019091030124
:1011A0000E9496210E9415122FEF81EE94E02150AB
:1011B00080409040E1F700C0000063E580910201AB
:1011C000909103010E949821CF910C9415128438BC
:1011D000C1F40E94C52082FD66C067E480910201CF
:1011E000909103010E9496210E9415122FEF81EE2B
:1011F00094E0215080409040E1F700C0000067E497
:10120000DDCF8CEF8C0F813AF8F48C2F0E946E1F8B
:10121000811149C06C2F80910201909103010E94BD
:101220006021882349F06C2F809102019091030185
:101230000E9498210E9415126C2F809102019091BA
:1012400003010E949621C0CF80E28C0F883048F4C1
:10125000C77081E001C0880FCA95EAF70E94D611D5
:10126000B3CFEBE5EC0FE33040F4F0E0E95BFE4F89
:10127000808190E0CF910C942821E8E5EC0FE731D4
:1012800050F4F0E0EE0FFF1FE75EFE4F808191818A
:10129000CF910C943E21CD3E30F08C2F0E94B81897
:1012A000CF910C948A19CF910895882309F464C0D2
:1012B000823879F40E94C52081FF5EC069E3809185
:1012C0000201909103010E9496210E94151269E388
:1012D00010C08338B1F40E94C52080FF4DC063E583
:1012E00080910201909103010E9496210E941512A3
:1012F00063E580910201909103010E9498210C9472
:101300001512843879F40E94C52082FF35C067E445
:1013100080910201909103010E9496210E94151272
:1013200067E4E7CF9CEF980F913A10F4682FE1CF74
:1013300090E2980F983050F4877091E001C0990FB7
:101340008A95EAF7892F0E94DC11D9CF9BE5980F87
:10135000933020F480E090E00C94282198E5980FD9
:10136000973120F480E090E00C943E218D3E20F0F7
:101370000E9413190C948A1908951F93CF93DF9339
:10138000182FEB010E94A608209741F08FE99FE0FB
:101390000197F1F700C000002197F6CF812FDF9170
:1013A000CF911F910C945509893319F060E070E0DA
:1013B00002C060E570E00C94BD09882321F00E9412
:1013C000D6110C9415120895882321F00E94DC1187
:1013D0000C9415120895CF92DF92EF92FF920F9323
:1013E0001F93CF93DF937C01D62FC72FFC0112816F
:1013F000058102950F700E94CC118823B9F011234A
:10140000A9F08C2F807F803421F080E28D0F88300E
:1014100068F08091CC0282FD09C082E00E947512C2
:101420000E94CC1191E0D82ED92601C0D12CCC2E0F
:10143000C2948FE0C8228C2D90E08C30910508F08A
:10144000CFC1FC01EA5AFF4F0C94572A8C2F807FA2
:10145000CF70882311F0C295C07F112399F0CC235F
:1014600009F4AAC180E28D0F883010F0D11104C0B8
:101470008C2F0E94D61103C08C2F0E94E6110E946F
:1014800015129AC18D2F0E945509CC2309F4A8C1C9
:1014900080E28D0F883038F1DD2329F18C2F0E94F6
:1014A000EC1124C08C2F807FCF70803211F0C29558
:1014B000C07FDD2319F0D130A1F13DC08091CC0275
:1014C00082FF17C0112349F0CC2329F08C2F0E94F2
:1014D000D6110E94151280E070C180E00E9455096B
:1014E000CC2309F47DC18C2F0E94DC110E941512BF
:1014F00077C1112371F0002341F0013031F40E94D3
:10150000F6118C2B0E94FE116BC10E94F6118C2BE0
:101510001DC0002319F0013009F462C10E940B12B2
:1015200025C0112321F0063008F05AC10EC0053045
:1015300008F056C11BC0112361F0002331F0F70100
:10154000858180FF39C18F7085838C2F0E94DD09D2
:1015500047C1002359F0D93309F03FC1FFEF07EE2F
:1015600013E0F15000401040E1F735C18C2F0E948C
:10157000E40936C18C2F86958695837019F08130E9
:1015800061F02EC1112321F08D2F9C2F937002C08A
:1015900080E090E00E9428212BC1112321F08D2FA3
:1015A0009C2F937002C080E090E00E943E2120C1F9
:1015B0008D2F112319F00E94B81802C00E94131930
:1015C0000E948A1915C18C2F837009F047C0111130
:1015D0000BC12D2F229526952770220F220F6D2FDC
:1015E0006F70862F90E0A0E0B0E0022E04C0880F5C
:1015F000991FAA1FBB1F0A94D2F7D4FF10C04FE057
:1016000050E060E070E004C0440F551F661F771F74
:101610002A95D2F7409550956095709503C040E0AB
:1016200050E0BA01C695C695C3708A019B01082B8C
:10163000192B2A2B3B2BC901B801C23049F058F4B1
:10164000C13019F00E94EC0CCFC00E94DA0CCCC063
:101650000E94FE0CC9C00E94D80CC6C0112319F00C
:101660008C2F817001C08695882309F4BDC02D2F71
:10167000229526952770220F220F6D2F6F70862FCF
:1016800090E0A0E0B0E0022E04C0880F991FAA1FCE
:10169000BB1F0A94D2F7D4FF10C04FE050E060E0C7
:1016A00070E004C0440F551F661F771F2A95D2F7BC
:1016B000409550956095709503C040E050E0BA01A8
:1016C000C695C695C3708A019B01082B192B2A2B3E
:1016D0003B2BC901B801C23049F058F4C13019F0B0
:1016E0000E94B10D81C00E949F0D7EC00E94C30D5B
:1016F0007BC00E94120D78C0CF70112339F08C2F5F
:101700000E94380D8D2F0E94DD096EC08D2F0E9422
:10171000E4098C2F0E94590D67C0D23F21F128F4B3
:10172000D03F41F0D13FC1F043C0D33F19F1D43F86
:1017300079F03EC0112341F0053008F051C08C2FE4
:101740008F710E947E0D4CC0063008F049C0F7CF63
:101750008091CC0282FF18C0112339F08C2F8F7139
:101760000E94380D3DC01123C9F38C2F8F710E9448
:10177000590D36C0112329F08C2F8F710E94230D33
:101780002FC00E941E0D2CC0112349F0CF718C2F49
:101790000E94380D63E08C2F0E945A1221C081E014
:1017A0000E9475120230E0F082E00E94751218C0AB
:1017B000112331F0002391F28D2F0E94A60810C052
:1017C000002399F2D93349F41FEF27EE33E011508B
:1017D00020403040E1F700C000008D2F0E945509E5
:1017E00088EF8C0D843020F40E94C5200E941408DC
:1017F000DD20C9F00E94C81180FD15C0F7011282DA
:101800000E94C2110E94380DC7010E94340C0E9430
:10181000C211DF91CF911F910F91FF90EF90DF9058
:10182000CF900C94590DDF91CF911F910F91FF90A4
:10183000EF90DF90CF9008950F931F93CF93DF9396
:10184000EC01688179818A810E947A0E8C010E9464
:10185000D50D0E94C60CB801CE010E94EB09DF91A4
:10186000CF911F910F910895CF93DF93EC01988151
:1018700089812B813C81232B31F08F3F31F481E032
:101880009F3F19F403C081E001C080E080FD1DC0CE
:10189000CE010E946E07811110C00E94CC118823D6
:1018A000A1F08A81882389F08091CC0282FD0DC04D
:1018B00082E0DF91CF910C947512CE010E941C0C36
:1018C000CE01DF91CF910C944F07DF91CF91089516
:1018D00080E090E00E94282180E090E00E943E217C
:1018E0000E94F3110E9415120E943D1B0C948A194C
:1018F00080910201909103010E949A210C94680C3E
:101900000E94E3110C94780C92959F70963079F0B8
:1019100010F4925001C09A50923068F4803F69F000
:1019200018F4883E40F409C0843F29F406C0883E7C
:1019300020F0813F11F080E0089581E00895FC01DE
:10194000808191810E946F0E0E94840C0895CF9334
:10195000DF9300D000D01F92CDB7DEB70F900F906D
:101960000F900F900F90DF91CF910895CF93DF9359
:1019700000D000D000D0CDB7DEB726960FB6F894D1
:10198000DEBF0FBECDBFDF91CF91089508950895BA
:101990000C94C70C0C94C80C0E94CA0C60933602BD
:1019A0007093370280933802909339020C94680C3C
:1019B0000C94CC0C0F931F930091360210913702B8
:1019C0002091380230913902602B712B822B932B9E
:1019D0001F910F910C94CC0C0F931F930091360222
:1019E000109137022091380230913902602371231F
:1019F000822393231F910F910C94CC0C0F931F9370
:101A0000009136021091370220913802309139024C
:101A100060277127822793271F910F910C94CC0C7C
:101A20000C94C70C0E94100D609332027093330225
:101A300080933402909335020C94680C60E070E05F
:101A4000CB010C94120D0F931F9341E050E060E026
:101A500070E08A019B0104C0000F111F221F331F79
:101A60008A95D2F7C901B8011F910F910C94120DFC
:101A70000F931F9341E050E060E070E004C0440F1A
:101A8000551F661F771F8A95D2F780913202909179
:101A90003302A0913402B09135028A019B01082BD8
:101AA000192B2A2B3B2BC901B8011F910F910C94C4
:101AB000120D0F931F9341E050E060E070E004C00E
:101AC000440F551F661F771F8A95D2F74095509592
:101AD000609570958091320290913302A09134020A
:101AE000B09135028A019B01082319232A233B2345
:101AF000C901B8011F910F910C94120D0F931F9300
:101B000041E050E060E070E004C0440F551F661FE4
:101B1000771F8A95D2F78091320290913302A0917B
:101B20003402B09135028A019B01082719272A2720
:101B30003B27C901B8011F910F910C94120D0F930F
:101B40001F930091320210913302209134023091A0
:101B50003502602B712B822B932B1F910F910C94CC
:101B6000120D0F931F9300913202109133022091B6
:101B700034023091350260237123822393231F9115
:101B80000F910C94120D0F931F930091320210913C
:101B90003302209134023091350260277127822769
:101BA00093271F910F910C94120D08952FE0929F8F
:101BB000800D1124E82FE695E695E695877051E0B3
:101BC00001C0550F8A95EAF785E0E89FF0011124DE
:101BD000E050FE4F20E030E070E04081CB01022E6B
:101BE00002C0969587950A94E2F7817081958427C3
:101BF0008523842781932F5F3F4F2530310569F777
:101C000008952FE0929F800D1124682F66956695A8
:101C10006695982F977085E0689FB001112440E089
:101C200050E080E0FB01E40FF51FE050FE4F208103
:101C300030E0092E02C0369527950A94E2F721700C
:101C40003327042E01C0220F0A94EAF7822B4F5F3C
:101C50005F4F4530510531F70895BF92CF92DF9223
:101C6000EF92FF920F931F93CF93DF938C01C0905D
:101C70003202D0903302E0903402F090350280912D
:101C8000360290913702A0913802B0913902C82AE9
:101C9000D92AEA2AFB2ACFE1D0E0D701C6010C2ECF
:101CA00004C0B695A795979587950A94D2F780FDBD
:101CB00004C0219790F7B12C07C0BC2EB8018C2F1F
:101CC0000E9484150197A9F38B2DDF91CF911F916D
:101CD0000F91FF90EF90DF90CF90BF900895CF933A
:101CE000DF93EC010E942D0EBE010E948415DF914E
:101CF000CF9108951F93CF93DF93EB019091FF0154
:101D0000992321F0CB010E946F0E13C0882349F064
:101D1000CB010E942D0E182F682FCE010E94D60DE8
:101D200004C0CB010E94010E182FBE01812F0E941A
:101D30008415DF91CF911F9108951F93CF93DF9367
:101D4000C0913A0216E080913B02C81799F0D0E0AA
:101D50001C9FF0011D9FF00D1124E45CFD4F40819C
:101D6000518162817381848195810E94B60C219694
:101D7000C770E9CFDF91CF911F91089540916C0218
:101D800050916D0260916E0270916F0280917002AD
:101D9000909171020C94B60CEF92FF920F931F93E7
:101DA000CF93DF938091710282958F7009F065C0A7
:101DB00080916E02882309F460C080913A02F0900D
:101DC0003B0210916C0200916D0260916F02709164
:101DD000700291E01F3F09F090E0C0910001D091A6
:101DE0000101292F96E0E92E8F1509F446C06115EF
:101DF000710521F00F3F21F030E003C031E001C058
:101E0000322F90E030FD36C0E89EF001E99EF00DE3
:101E10001124DF01A45CBD4F11963C911197301342
:101E200029C03C91311326C012963C911297311172
:101E300021C013964D915C911497461B570B4C177C
:101E40005D07C0F4809171028F7080618093710290
:101E5000EF5BFD4F80818F70806180838CE692E024
:101E60000E94340CDF91CF911F910F91FF90EF9062
:101E70000C949D0E01968770B7CFDF91CF911F9183
:101E80000F91FF90EF9008959F92AF92BF92CF92E3
:101E9000DF92EF92FF920F931F93CF93DF93CDB713
:101EA000DEB761970FB6F894DEBF0FBECDBF8C01D1
:101EB00085E0F801DE011D9601900D928A95E1F70B
:101EC000D8011296EC9090916C02E0916D022091F5
:101ED0006F02309170022115310531F0EF3F31F47E
:101EE00081E09F3F19F403C081E001C080E0B82F7A
:101EF000B1709B2E80FD47C1D8014C9111965C9129
:101F000011971396AD90BC9014978CE6C82E82E082
:101F1000D82EF0906E02B501621B730B2091000168
:101F200030910101FF2009F4D9C08091710262173C
:101F3000730708F095C0282F207F09F052C05E1368
:101F400013C0491311C0FE2CE1100EC08F708061C8
:101F5000809371020E94BE0EC6010E94340C8091D3
:101F60007102F80185834DC1AB2831F05F3F31F438
:101F700081E04F3F19F403C081E001C080E080FDA3
:101F800003C081E08E2502C080E090E0F82FF17060
:101F9000FF2E80FF1CC080913A0220913B0236E068
:101FA000821709F40BC190E0389FF001399FF00DC2
:101FB0001124E45CFD4F6181561306C06081461315
:101FC00003C06281E61203C001968770E9CFFE2C40
:101FD000EE2009F416C18091710281608093710234
:101FE00054C05E1306C0491304C0E11002C0F801DA
:101FF00099C0C8010E949F0C882361F1EE2051F125
:1020000020917102822F82958F7090E0029774F078
:1020100080916C0290916D0298878F831986BB86A0
:10202000AA862C87CE0107960E94340C86E0F80120
:10203000ACE6B2E001900D928A95E1F70E94CC0ED9
:102040000E94BE0E0AC05E1711F1C8010E949F0CCB
:1020500081112CC0C8010E94340CFF24F394D1C01C
:10206000282F207F81F77A2DB98AA88A6E2D898939
:102070000E94A70C8CE692E00E94340C86E0D60108
:102080001D928A95E9F70E94BE0EF12CBAC0491341
:10209000DCCFE110DACFF8018583C8010E94340C4F
:1020A00086E0D6011D928A95E9F7ABC0EE2091F249
:1020B00020917102822F82958F7090E002970CF42C
:1020C000B5CF80916C0290916D029A8389831B82B7
:1020D000BD82AC822E83CE010196A6CF6217730714
:1020E00008F044C0FE2CEE2009F4B4CF5E1330C0DB
:1020F00049132EC02091710220FD21C0822F8295AC
:102100008F70482F50E041155105C9F0F801258323
:102110004F30510541F08F5F982F9295907F822F1D
:102120008F70892B8583C8010E94340C86E0F801EA
:10213000ACE6B2E001900D928A95E1F73CC086E0F2
:10214000F801ACE6B2E001900D928A95E1F759C032
:10215000C8010E949F0C811169CF8091710281603A
:1021600080937102C8010E94340C4BC07A2DB98A49
:10217000A88A6E2D89890E94A70C86E0D6011D923F
:102180008A95E9F718C0EE2009F464CFC8010E94CF
:102190009F0CF82E882309F45DCF86E0F801ACE6A9
:1021A000B2E001900D928A95E1F78CE692E00E94F0
:1021B000A0080E94CC0E0E94BE0E23C04D875E87F1
:1021C0008D859E850E946F0E292F22952F702230BB
:1021D00028F49F7039F0811105C00BC0243028F419
:1021E0009F7049F4805E883020F0C8010E94340C52
:1021F0009F2CF92C06C0D80115969C91907F91F7E1
:10220000F8CF8F2D61960FB6F894DEBF0FBECDBF0D
:10221000DF91CF911F910F91FF90EF90DF90CF90C2
:10222000BF90AF909F9008951F93CF93DF93CDB74A
:10223000DEB72C970FB6F894DEBF0FBECDBF4F832D
:10224000588769877A878B879C87CE0107960E947B
:10225000440F8823D1F09F8188852A853B85232BD5
:1022600031F08F3F31F481E09F3F19F403C081E0EA
:1022700001C080E080FD47C04F81588569857A851F
:102280008B859C850E94B60C3EC086E0FE01379689
:10229000DE01119601900D928A95E1F7FF81E885A4
:1022A0006A857B856115710531F0EF3F31F481E07E
:1022B000FF3F19F403C081E001C080E080FD23C02E
:1022C00020913B0230E0C901019687709927409127
:1022D0003A0250E084179507F1F1F983EA837D8390
:1022E0006C8396E0929FD001939FB00D1124A45C63
:1022F000BD4FFE01319601900D929A95E1F78093C2
:102300003B020E949D0E16E080913A0290913B02A2
:10231000891771F1189FC0011124845C9D4F0E94A0
:10232000440F882329F1E0913A021E9FF001112405
:10233000E45CFD4F4081518162817381848195818C
:102340000E94B60C80913A0290E00196877099271E
:1023500080933A02D9CF0E94800C10923B021092D7
:102360003A02ECE6F2E086E0DF011D928A95E9F799
:102370002C960FB6F894DEBF0FBECDBFDF91CF9184
:102380001F91089580917A02859585958595089588
:1023900080917A028770089590917A02977081E017
:1023A00009F480E008958091850208959091850256
:1023B000892B8093850208958095909185028923C9
:1023C0008093850208951092850208959091840269
:1023D000892B8093840208958095909184028923AB
:1023E00080938402089510928402089580917B0264
:1023F000089508950C94F9110C94FA119091CC025F
:1024000092FD08C090917B02981721F080937B0287
:102410000C94FC11089580917B02882329F010927E
:102420007B0280E00C94FC110895CF93DF93E09140
:102430000201F0910301809185028083E091020105
:10244000F0910301908180918402892B8083809197
:102450007B02882381F0E0910201F09103019081D9
:10246000892B808380910201909103010E94542165
:1024700081110E940B12C0910201D091030148E02A
:1024800050E062E772E0CE010E94712A892B69F068
:1024900088E0FE01A2E7B2E001900D928A95E1F793
:1024A000CE01DF91CF910C94D120DF91CF9108958F
:1024B0000C94F9119091CC0292FD10C098E0899F84
:1024C00090011124262B20937A020E94380D8091CE
:1024D0007A028595859585950C9458120C94380D43
:1024E00010927A0280E00C94581220917A02809522
:1024F000822380937A02982F977099F430E0482FC6
:10250000082E000C550B2417350759F09091CC027A
:1025100092FD07C08595859585950E94590D0C946F
:1025200070120895CF939091CC0292FB222720F94C
:102530002817F9F0C82F892FC0FB82F98093CC02AD
:102540008091CB029091CC020E94EE1282E00E9418
:1025500075128091980280FF0CC01F92CF9385E680
:1025600093E09F938F930E94FF060F900F900F9020
:102570000F90CF9108958091CC0282FB882780F93B
:1025800091E089270C94921281E00C94921280E0E1
:102590000C94921280E090E00E94862A21E0893E0D
:1025A0009E4F09F020E0822F089582E090E00C9485
:1025B0007E2A83E090E00C947E2ACF9384E090E022
:1025C0000E947E2AC82F82E290E00E947E2A2C2F51
:1025D00030E0A901582BCA01CF910895CF93C92F9C
:1025E000682F84E090E00E948C2A6C2F82E290E0B9
:1025F000CF910C948C2AAB01BC018FE090E00C943D
:102600009E2AAB01BC0183E190E00C949E2A60E01D
:1026100070E0CB010C94011360E070E0CB010E94EC
:10262000FB120C94071369EE7EEF80E090E00E94AD
:10263000AA2A60E082E090E00E948C2A60E083E0B9
:1026400090E00E948C2A109236021092370210926B
:1026500038021092390260E084E090E00E948C2AF7
:1026600060E082E290E00E948C2A60E085E090E0E9
:102670000E948C2A60E086E090E00E948C2A6FEF36
:1026800087E090E00E948C2A40E050E0BA0188E0A8
:1026900090E00E949E2A60E08DE090E00E948C2AEB
:1026A00040E050E0BA0188E190E00E949E2A60E09C
:1026B00087E190E00E948C2A40E050E0BA018CE172
:1026C00090E00E949E2A60E070E080E290E00E942C
:1026D000AA2A40E050E0BA0188E190E00E949E2AD8
:1026E0000C940C130C941313682F8EE090E00C9450
:1026F0008C2A0E94492260939402709395028093E1
:102700009602909397026093900270939102809347
:10271000920290939302089585B7806885BF85B72C
:10272000806885BF089581E008950C9493130895FF
:102730000C9497130C9497130C949A130C9497136E
:102740000C949E130C9497130E948C1381E894E2CE
:102750000E94BB200E94A2130C94A0130E94981305
:102760000C9497130E9461160C9413080E94342253
:102770000E948C170E94B2130C949C135F926F926C
:102780007F928F929F92AF92BF92CF92DF92EF9201
:10279000FF920F931F93CF93DF93CDB7DEB72A97A6
:1027A0000FB6F894DEBF0FBECDBF0E94A117C82E92
:1027B00081110E94791336E8832E32E0932E00E0D7
:1027C00010E0502E802F0E9485165C01F40161906C
:1027D00071904F016826792661147104B1F40F5F7E
:1027E0001F4F0530110569F78FEF89838A831B829C
:1027F0000E943D228160782F9D838C8349815A817C
:102800006B818D810E9456083AC08091980281FDAB
:102810000E948E16D12CEE24E394F12CC3018E215C
:102820009F21892B29F10E9495138823A9F0DE822C
:102830005F82AE20BF2081E0AB2809F480E088876A
:102840000E943D228160782F9A8789874E815F811F
:1028500068858A850E945608000F111FF801EA5703
:10286000FD4F80819181E826F926F182E08207C040
:10287000D394EE0CFF1CFFE0DF12D0CFB0CF81E08D
:10288000C11001C080E02A960FB6F894DEBF0FBEDB
:10289000CDBFDF91CF911F910F91FF90EF90DF900F
:1028A000CF90BF90AF909F908F907F906F905F90F0
:1028B00008950E94BE130E942A1A0C942408CF93F4
:1028C000DF930E948915EC01811521E5920708F03C
:1028D00045C0811530E5930708F094C0883E910506
:1028E00028F5803E910508F0F8C0883A910570F40B
:1028F000853A910508F07CC08130910509F475C0D6
:1029000008F4E8C0049708F0E8C0E4C08F3B9105E4
:1029100008F0E0C0C85AD0E0CC0FDD1FC65BDE4F28
:102920000990D881C02DCE019464D8C0811540E2B1
:10293000940758F4811551E0950708F0CEC08D3EFC
:10294000910508F4C7C09065C9C0C11580E4D807D7
:1029500008F4C0C0DF70CE01906AC0C0811525E5C3
:102960009207A8F4811534E5930708F095C0811506
:1029700043E5940708F07BC0811552E5950708F000
:1029800061C0D82FCC27CE01816F906AA7C0C11536
:1029900089E5D807A0F4C11528E5D20708F082C060
:1029A000C11536E5D30708F095C08C2F0E941D167F
:1029B0008F7190E0D82FCC27CE0190628FC0C115C7
:1029C0004AE5D40708F474C0CE01905681159042B0
:1029D00008F080C08D2F8F710E941D16DD27D062F8
:1029E0008F71AE01582BCA0179C081E090E076C0AA
:1029F000C55AD0E0C858DE4F8881C82FD0E0CE013C
:102A000090646CC074E0969587957A95E1F7282FCD
:102A100023703C2F337081E090E002C0880F991F33
:102A20003A95E2F79C68AC01522B9A019C2F9F705B
:102A30009695969550E2959FE0011124C9018C2B43
:102A40009D2B4CC08370992721E030E002C0220FFB
:102A5000331F8A95E2F79C2F9695969580E2989F72
:102A6000E0011124C22BD32BCE019C6837C08370A8
:102A7000992721E030E002C0220F331F8A95E2F748
:102A80009C2F9695969540E2949FE0011124C22BCD
:102A9000D32BCE019A6822C0D82FCC27CE01846FC9
:102AA000906A1CC0DC2FCC27CE01806F906A16C0C4
:102AB0008C2F8F700E941D1694E0D695C7959A951D
:102AC000E1F7CF70D0E0DC2FCC27D0699E01282B16
:102AD000C90104C080E090E001C0CE01DF91CF9138
:102AE00008952BE4829FC0011124FC012FE0729F06
:102AF000E00DF11D1124E60FF11DEE0FFF1FE8524E
:102B0000FF4F8591949108950E9471150E945F1462
:102B100008958238910569F1B0F48133910509F483
:102B20006DC048F48932910509F463C08A32910579
:102B300009F469C008958533910509F455C08933B6
:102B40009105B9F00895833E910569F138F4803E0E
:102B50009105B1F0823E910509F10895863E9105F7
:102B6000A9F1873E9105B9F1843E910509F064C051
:102B700023C02091CB0220FD4FC021FD4DC0089500
:102B80008091CB0280FD44C08091CC0280FF44C084
:102B90008091CB0284FD42C083EE4DC08091CB0278
:102BA00082FF38C0F5CF8091CB0282FD33C0809187
:102BB000CC0280FD31C0ECCF8091CC0281FF32C0CD
:102BC0008091CB0284FD2AC087EE35C08091CB0274
:102BD00083FF26C0F5CF8091CB0283FD21C0809179
:102BE000CC0281FD1FC0ECCF8091CB0285FD1CC0C3
:102BF0001DC08091CB0285FD19C016C08091CB020B
:102C000086FD16C017C08091CB0286FD13C010C090
:102C100089E311C082EE0FC080EE0DC080E00BC0D2
:102C200086EE09C084EE07C089E205C085E303C0D3
:102C30008AE201C081E390E008959091CB0292FF77
:102C40000DC0282F2871283019F4877F846006C0B2
:102C5000282F2471243011F48B7F886093FF0DC0DE
:102C6000282F2871283119F4877E846106C0282F07
:102C70002471243111F48B7E88612091CC0220FFD5
:102C80000DC0382F3871383019F4877F816006C045
:102C9000382F3171313011F48E7F886021FF0DC0E3
:102CA000282F2871283119F4877E816106C0282FCA
:102CB0002171213111F48E7E886194FD877E089503
:102CC00008950E94CA12811102C00E9472130E94CC
:102CD000D512809398020E94DD129093CC028093CB
:102CE000CB020E9460160E94D912682F70E080E02B
:102CF00090E00E94D80C6091320270913302809172
:102D00003402909135020C94100DE82FF0E0EE0F94
:102D1000FF1FE952FD4F808191810895CF92DF928C
:102D2000EF92FF920F931F93CF93DF938AE893E084
:102D30000E94660687EDE82E82E0F82EC0E0D0E023
:102D400095E8C92E93E0D92E0CE713E0DF93CF93DB
:102D5000DF92CF920E94FF0682E893E00E9466060F
:102D6000F701819191917F010E94F9079F938F93C1
:102D70001F930F930E94FF068AE793E00E94660666
:102D800021968DB79EB708960FB6F8949EBF0FBEDA
:102D90008DBFC530D105D1F6DF91CF911F910F9135
:102DA000FF90EF90DF90CF90089580EA8A95F1F739
:102DB000089500C008950C94D51608950C94DD165E
:102DC0000C94DE160C94DD160C94E216F894E82FA1
:102DD000E295EF70F0E031A1282F2F7081E090E0B4
:102DE00001C0880F2A95EAF7982F9095932391A315
:102DF00092A1892B82A3789408950F931F93CF9368
:102E0000DF93CAE8D1E089918F3F11F00E94E61666
:102E100081E0CF38D807B9F7CBE7D1E00AE811E075
:102E200089918F3F11F00E94E6160C171D07C1F71C
:102E3000DF91CF911F910F910895BF92CF92DF92B2
:102E4000EF92FF920F931F93CF93DF938C01C62FC6
:102E5000D0E0CE0186579E4F6C01FC0190819F3FD0
:102E600009F450C0B62EF894E92FE295EF70F0E027
:102E700081A19F7021E030E001C0220F9A95EAF70E
:102E8000822B81A382A12095282322A378940E94DB
:102E9000D916EBE7F1E04AE851E021E030E0E12C1F
:102EA000F12C61916F3F89F0A62FA295AF70B0E031
:102EB00090968C9190E06F7002C0959587956A9579
:102EC000E2F780FD02C0C90102C080E090E0E82A7C
:102ED000F92A220F331F4E175F0719F7F601808179
:102EE0008F3F11F00E94E61661E0E114F10409F44D
:102EF00060E08B2D0E94DB16CC0FDD1FC00FD11FB1
:102F0000F982E882DF91CF911F910F91FF90EF90AE
:102F1000DF90CF90BF9008950E94FD168AE0E7ED04
:102F2000F2E0DF01982F1D929A95E9F7EDECF2E0BF
:102F3000DF011D928A95E9F785E00E94EC170C9459
:102F40005A07FF920F931F93CF93DF93CDB7DEB74E
:102F50002A970FB6F894DEBF0FBECDBF8E010F5F6C
:102F60001F4F8AE0F80111928A95E9F7F12C6F2D35
:102F7000C8010E941D17F394F5E0FF12F8CF4AE054
:102F800050E0B8018DEC92E00E94712AFF24F39486
:102F9000009709F4F12C892B41F08AE0F801ADEC9F
:102FA000B2E001900D928A95E1F72F2D45E067ED93
:102FB00072E08DEC92E00E94ED170E945C078F2D6D
:102FC0002A960FB6F894DEBF0FBECDBFDF91CF912A
:102FD0001F910F91FF9008950895FF920F931F93F3
:102FE000CF93DF93F82E092F162FD72FC42F22232C
:102FF00049F081E080939B020E943D2290939A02C7
:103000008093990280919B028823D9F08091990244
:1030100090919A020E945522059798F0EF2DF02F7B
:10302000A12FBD2F80E090E04C2F50E08417950732
:1030300034F4219131912D933D930196F7CF109265
:103040009B02DF91CF911F910F91FF9008950E94F5
:10305000FD240E94B6130C9409250E940D250E94A0
:1030600059140C942B250E94DB210E94E4240E9419
:10307000A4130E9427180E942D180E94AE13FBCFA4
:103080008091A20280FF06C06091090170E0660F86
:10309000771F26C081FF04C06091090184E005C04C
:1030A00082FF07C06091090188E0689FB001112488
:1030B00017C09091A1029923D1F060910801961751
:1030C00088F72091090188E0289F90011124929FA0
:1030D000A001939F500D112470E0CA010E94432A61
:1030E0006038710540F46115710519F406C068E097
:1030F00070E0862F08958FE7089581E0089580910C
:10310000A20280FF08C06091050170E07595679587
:103110007595679521C081FF06C06091050170E03B
:103120007595679519C082FF04C06091050170E034
:1031300010C09091A002992399F060910401961714
:10314000A0F780910501899FC001112470E00E94C1
:10315000432A6038710540F46115710519F406C001
:1031600061E070E0862F08958FE7089581E008956B
:103170008D3E21F40E944018819504C08E3E29F4B2
:103180000E9440188093A60208958F3E21F40E9469
:103190004018819504C0803F29F40E944018809314
:1031A000A5020895893F19F40E947F1805C08A3F3F
:1031B00031F40E947F1881958093A70208958B3F78
:1031C00021F40E947F18819504C08C3F29F40E944D
:1031D0007F188093A80208959FE0980F983078F4A4
:1031E00021E030E0A90102C0440F551F9A95E2F793
:1031F000CA019091A402892B8093A40208958D3F67
:1032000021F48091A20281600BC08E3F21F4809155
:10321000A202826005C08F3F29F48091A2028460DF
:103220008093A20208958D3E39F49091A60297FFF3
:1032300035C01092A60259C08E3E29F49091A60284
:103240001916BCF32BC09091A5028F3E29F497FF6D
:1032500025C01092A50249C0803F19F41916CCF37D
:103260001DC09091A702893F29F41916BCF4109251
:10327000A7023BC08A3F19F497FF10C0F8CF8B3FDD
:1032800039F49091A80297FF09C01092A8022DC0AE
:103290008C3F21F49091A8021916BCF39FE0980F7F
:1032A000983080F421E030E0A90102C0440F551F9E
:1032B0009A95E2F7CA0180959091A40289238093A0
:1032C000A40213C08D3F21F48091A2028E7F0BC017
:1032D0008E3F21F48091A2028D7F05C08F3F29F49B
:1032E0008091A2028B7F8093A2028091A50281111E
:1032F00006C08091A602811102C01092A1028091A5
:10330000A702811106C08091A802811102C010920B
:10331000A00208958091980283FF7EC088EC93E01C
:103320000E9466068091A4021F928F9383EC93E023
:103330009F938F930E94FF0681EC93E00E946606A4
:103340008091A502282F082E000C330B3F938F93FA
:103350008EEB93E09F938F930E94FF068CEB93E09C
:103360000E9466068091A602282F082E000C330BBF
:103370003F938F9389EB93E09F938F930E94FF0677
:1033800087EB93E00E9466068091A702282F082E03
:10339000000C330B3F938F9384EB93E09F938F93B9
:1033A0000E94FF0682EB93E00E9466068091A802CD
:1033B000282F082E000C330B3F938F938FEA93E056
:1033C0009F938F930E94FF068CEA93E00E9466060B
:1033D0008091A1021F928F9389EA93E09F938F932C
:1033E0000E94FF0687EA93E00E9466068091A2028F
:1033F0001F928F9384EA93E09F938F930E94FF061E
:1034000081EA93E00E9466068DB79EB74C960FB690
:10341000F8949EBF0FBE8DBF0E943D222091A50251
:10342000211104C02091A602222321F090939F0233
:1034300080939E022091A702211104C02091A8022E
:10344000222321F090939D0280939C0283EA92E0D4
:103450000C941A21EF92FF920F931F93CF93DF9357
:1034600000D000D000D0CDB7DEB786E0E3EAF2E0CE
:10347000DE01119601900D928A95E1F7E090A50288
:10348000F090A6020091A7021091A8021092A50246
:103490001092A6021092A7021092A802E11003C097
:1034A000FF2009F45DC080919E0290919F020E94CE
:1034B0005522AC019091A102992339F020910A0183
:1034C00030E02417350758F04BC020910B018AE0FB
:1034D000289F900111242417350718F041C09F3F01
:1034E00019F09F5F9093A102EE2061F00E944018B6
:1034F0001E1414F09FEF01C091E0989F902D1124AD
:103500009093A502FF2061F00E9440181F1414F050
:103510009FEF01C091E0989F902D11249093A602F7
:103520003091A5023323E1F02091A6022223C1F0BD
:1035300045EB3403C0011124992319F09093A5029F
:1035400003C081E08093A50235EB2303C001112461
:10355000992319F09093A60203C081E08093A602FC
:10356000011103C0112309F45DC080919C02909168
:103570009D020E945522AC019091A002992339F03E
:103580002091060130E02417350758F04BC02091F8
:1035900007018AE0289F900111242417350718F0AD
:1035A00041C09F3F19F09F5F9093A002002361F0FC
:1035B0000E947F18101614F09FEF01C091E0989FB1
:1035C000902D11249093A702112361F00E947F187F
:1035D000111614F09FEF01C091E0989F902D1124D7
:1035E0009093A8023091A7023323E1F02091A80222
:1035F0002223C1F045EB3403C0011124992319F0B3
:103600009093A70203C081E08093A70235EB2303C8
:10361000C0011124992319F09093A80203C081E0FE
:103620008093A8028091A50281110BC08091A6020F
:10363000811107C08091A702811103C08091A80267
:1036400081110E948A19EB82FC820D831E8386E021
:10365000FE013196A3EAB2E001900D928A95E1F75E
:1036600026960FB6F894DEBF0FBECDBFDF91CF9187
:103670001F910F91FF90EF900895E3EAF2E086E04A
:10368000DF011D928A95E9F71092A1021092A00223
:103690001092A2020895CF93DF93EC01FB01828187
:1036A000882309F43CC1C430FDE5DF0760F4CB3F5B
:1036B0009CE5D90788F49E0122503C452431310510
:1036C00008F02EC109C0C236EDE5DE0729F0C63A82
:1036D000FDE5DF0709F024C10E94DD129093CC02C2
:1036E0008093CB02C1318CE5D80709F4C6C008F03D
:1036F00042C0C930ECE5DE0709F49BC000F5C530D7
:103700008CE5D80709F485C078F4C330ECE5DE0712
:1037100009F478C008F07AC0C230DC4509F0F5C081
:103720008091CB028160EFC0C7309CE5D90709F4D6
:1037300078C008F07AC08091CB028061E4C0CD30BF
:10374000FCE5DF0709F487C058F4CB309CE5D907C6
:1037500009F479C008F07BC08091CB0288606FC00B
:10376000CF30FCE5DF0709F480C008F082C080910B
:10377000CB02877FC8C0CE3F9CE5D90709F471C052
:1037800000F5C531FCE5DF0709F485C068F4C331F5
:103790009CE5D90709F475C008F095C00E94800C1B
:1037A0008091CB028F77AFC0CC3FFCE5DF07A9F15A
:1037B00008F054C0CB3FDC4509F0A7C08091CC0293
:1037C00040C0C230EDE5DE0709F489C058F4C115E8
:1037D0008DE5D80709F45AC008F069C08091CC0281
:1037E00082602FC0C236EDE5DE0709F47CC0C63A20
:1037F000FDE5DF0709F481C0C330DD4509F085C070
:1038000080E06EC08091CB0282607DC08091CB024F
:1038100016C08091CB02886076C08091CC02826015
:103820004FC08091CB0280626EC08091CB028064D9
:103830006AC00E94800C8091CB02806864C0846062
:1038400062C081603DC08091CB028E7F5CC0809160
:10385000CB028D7F58C08091CB0216C08091CC02E4
:1038600018C08091CC028D7F2BC08091CB028F7EBF
:103870004AC08091CB028F7D46C08091CB028F7B66
:1038800042C08091CB02877F8B7F3DC08091CC026C
:103890008D7F8E7F15C08091CB0282FB222720F97D
:1038A00091E0922790FB82F990FB83F92CC08091E4
:1038B000CC02982F909591708E7F892B90FB81F987
:1038C0008093CC0222C00E94800C8091CB0287FBA7
:1038D000222720F991E0922790FB87F914C081E01C
:1038E0000E94741312C08091CB0284FB222720F91E
:1038F00091E0922790FB84F906C08091CB02982F2B
:10390000909590FB80F98093CB028091CB029091AF
:10391000CC020E94EE120E94800C80E001C081E087
:10392000DF91CF910895809104011F928F93809130
:1039300005011F928F93809108011F928F938091B0
:1039400009011F928F9380910A011F928F9380919A
:103950000B011F928F938BEE93E09F938F930E94A6
:10396000FF068DB79EB70E960FB6F8949EBF0FBE9A
:103970008DBF0895883220F58E3108F068C08B30F5
:1039800091F1C0F4873009F0BEC081E080930B0153
:1039900084E180930A018AE0809309018EE180939B
:1039A000080188E08093050188E2809304018DE49A
:1039B00095E0C6C0833109F443C0843169F1A3C0E6
:1039C0008F3409F49EC028F4893231F1883359F0DC
:1039D0009AC0813531F008F4D4C0823509F4A7C00B
:1039E00092C08FEFA5C08FE695E00E9466060E9408
:1039F000931C1F9281E08F931F9288E08F9388E63B
:103A000094E09F938F930E94FF060F900F900F906A
:103A10000F900F900F9096C08CE695E00E9466067E
:103A20008091AD02882309F4AAC01092AD021092D1
:103A3000AC021092AB021092AA021092A902B1C07D
:103A40008EE595E00E9466060E94931C7BC08D5116
:103A50008093AD02833031F170F48130D1F0823047
:103A600009F03FC08AE091E09093AC028093AB02F2
:103A70008CE991E01FC0853059F108F1863089F555
:103A800084E091E09093AC028093AB0287ED91E0EB
:103A900011C08BE091E09093AC028093AB0283E97C
:103AA00091E008C089E091E09093AC028093AB0272
:103AB00088EA91E09093AA028093A90218C088E056
:103AC00091E09093AC028093AB0285EB91E0F2CF52
:103AD00085E091E09093AC028093AB0284EC91E09E
:103AE000E9CF1092AD028BE595E00E9466068091C9
:103AF000AD02882309F455C01F928F9387E595E0A6
:103B00000DC08AE015C08AE495E01AC097FF47C04F
:103B1000108280811F928F9384E495E09F938F930E
:103B20000E94FF060F900F900F900F900BC081E046
:103B3000E091AB02F091AC02309729F581E495E079
:103B40000E9466062091AD02222359F18091A902BC
:103B50009091AA02009711F48FE891E09F938F93C0
:103B60001F922F9388E395E09F938F930E94FF0607
:103B70000F900F900F900F900F900F9016C080E055
:103B8000089586EFD5CF2081082E000C990B820F67
:103B9000911D8F3F910509F00CF4B8CF8FEF808312
:103BA000B8CF84E395E00E94660681E00895CF9344
:103BB000C82F1F928F9385E895E09F938F930E9463
:103BC000FF0681E090E0A0E0B0E0BC01CD0104C0C0
:103BD000660F771F881F991FCA95D2F70E94D80CCD
:103BE0000F900F900F900F90CF910C94800CEF924C
:103BF000FF920F931F93CF93DF938B3109F4EDC0A6
:103C000008F08EC08B3009F4B1C008F078C086305F
:103C100009F4AFC020F4853009F4BDC04EC187302F
:103C200009F4C0C0883009F048C10E94D9121F921F
:103C30008F938AEB99E09F938F930E94FF060E94D7
:103C4000D51283FB992790F91F929F9382FB9927A6
:103C500090F91F929F9381FB992790F91F929F9350
:103C6000982F91701F929F931F928F9381E799E0F5
:103C70009F938F930E94FF060E94DD1287FB2227ED
:103C800020F91F922F9386FB222720F91F922F9352
:103C900085FB222720F91F922F9384FB222720F9EE
:103CA0001F922F9383FB222720F91F922F9382FBD1
:103CB000222720F91F922F9391FB222720F91F9290
:103CC0002F93292F21701F922F9381FB222720F9F8
:103CD0001F922F93282F21701F922F939F938F93C2
:103CE0008CE898E09F938F930E94FF068DB79EB754
:103CF00088960FB6F8949EBF0FBE8DBF35C0803139
:103D000009F495C020F48E3009F47BC0D6C086310A
:103D100009F4A8C0893109F0D0C085EF95E084C0CE
:103D20008A32E1F060F4873209F4C3C028F48E319E
:103D300008F4C3C08D51BEC0893269F1BEC083345E
:103D400048F48A3308F0B3C0853309F4B2C088332D
:103D500069F0B3C0833409F4ACC0AFC085E69AE023
:103D60000E9466060E947213C1E0ACC089EE96E024
:103D70005BC080919802817F8E7F8093980282EC55
:103D800096E00E94660681E69AE00E94660681E05F
:103D90008093AE02E9CF85E49AE00E9466060E9415
:103DA0005F07E2CF80919802C82FC095C170C0FB19
:103DB00080F980939802CC2329F089E39AE00E944D
:103DC000660680C08CE29AE00E94660680919802A6
:103DD000897F877F80939802C7CF9091980291FB4B
:103DE000CC27C0F981E0C827892FC0FB81F98093D7
:103DF0009802CC2319F08FE19AE029C081E19AE082
:103E000013C09091980292FBCC27C0F981E0C8279B
:103E1000892FC0FB82F980939802CC2319F082E0AD
:103E20009AE015C082EF99E00E9466069DCF9091BE
:103E3000980293FBCC27C0F981E0C827892FC0FBEB
:103E400083F980939802CC2351F086EE99E00E948A
:103E500066068091980281608093980233C089ED54
:103E600099E0E2CF0E944922162F072FF82EE92E63
:103E7000D091CA02C09118010E94C520EF92FF9212
:103E80000F931F931F92DF931F92CF931F928F93D5
:103E90008AE895E09F938F930E94FF068DB79EB7A7
:103EA0000C960FB6F8949EBF0FBE8DBF5DCF8953A1
:103EB00001C080E00E94D71D57CF87ED99E00E9496
:103EC0006606C0E08C2FDF91CF911F910F91FF907C
:103ED000EF90089580E008950C946A1FCF93C82F47
:103EE0008091AE02813071F040F0823009F045C01F
:103EF0008C2F0E94BA1C81E046C00E94D3118232EE
:103F0000F1F504C00E94D311823261F48C2F0E941B
:103F10006C1F811104C08C2F0E94F71D2CC081E002
:103F200090E029C08C2F0E946A1F811123C0C431E8
:103F3000C9F058F4CB3069F0C031B9F482E0809315
:103F4000AE0288E30E94BA1C15C0C93259F0C833CA
:103F500061F482EC96E00E94660681E895E00E949A
:103F6000660608C01092AE020CC08FE795E00E9472
:103F7000660607C081E0817006C01092AE0280E044
:103F800002C080E0F8CFCF910895CF93DF938631C0
:103F90009C4541F5EB010E94D311982F8A81209115
:103FA000020130910301882379F09A7A81E009F4C3
:103FB00080E08093AF02911102C069E201C065E325
:103FC000C9010E9496210AC08091AF02811102C0EE
:103FD00069E201C065E3C9010E9498210E9415129F
:103FE00080E001C081E0DF91CF9108950F931F938E
:103FF000CF93DF93C42FD22FFC0182818823C9F095
:104000004093B2020E943D229093B1028093B0028D
:1040100080E28C0F883008F057C0C77081E001C083
:10402000880FCA95EAF7DF91CF911F910F910C94F9
:10403000DD098091B202481330C08091B0029091A6
:10404000B1020E945522883C910538F510E21D0FFF
:10405000CD17B9F080E28C0F883040F4C77081E052
:1040600001C0880FCA95EAF70E94E409183028F5C4
:1040700081E09D2F977001C0880F9A95EAF70E9402
:10408000DD09802F0E94D4091830F0F4D77081E048
:1040900001C0880FDA95EAF70AC080E28C0F8830F9
:1040A00098F4C77081E001C0880FCA95EAF7DF91E4
:1040B000CF911F910F910C94E409802FDF91CF9144
:1040C0001F910F910C94D409DF91CF911F910F9103
:1040D00008950F939C01CB01243F4CE5340731F147
:1040E00088F4293DFCE53F07D9F02A3D4CE534072B
:1040F00079F1283D3C45A9F506E221EE41EE68ED57
:104100007CE52BC0263FFCE53F07E1F0A8F0273F08
:104110003C4539F507E225EE46EE67EF7CE51DC02C
:1041200007E225EE45EE69ED7CE517C006E221EEDB
:1041300040EE64EF7CE511C007E225EE44EE65EF4A
:104140007CE50BC006E221EE42EE66EF7CE505C0A1
:1041500008E221E045EE6AED7CE50E94F61F80E072
:1041600008C0FC018281882319F01092B20201C0BC
:1041700081E00F9108959093FD018093FC010895D3
:104180009093B8028093B7020895E091B702F0913E
:10419000B802309721F00190F081E02D099480E081
:1041A0000895EF92FF920F931F93CF93DF93E091C7
:1041B000B702F091B8023097B1F18C010280F3811F
:1041C000E02D09958091980282FF2DC080FF04C0E8
:1041D0008EE79AE00E946606E80118E088E7E82E7C
:1041E0008AE0F82E8091980280FF0BC088811F9290
:1041F0008F93FF92EF920E94FF060F900F900F9007
:104200000F90115021961111EDCF8091980280FFEF
:104210000AC086E79AE0DF91CF911F910F91FF903E
:10422000EF900C946606DF91CF911F910F91FF9054
:10423000EF900895E091B702F091B802309739F00D
:1042400022E0DC012C930480F581E02D099408958F
:104250002091B5023091B6022817390771F090937A
:10426000B6028093B502E091B702F091B8023097A0
:1042700021F00680F781E02D099408952091B30282
:104280003091B4022817390771F09093B4028093EB
:10429000B302E091B702F091B802309721F00084A8
:1042A000F185E02D09940895FC01329697E080E0B5
:1042B000915029F021912223D9F38F5FF9CF0895EE
:1042C000662349F0FC01329608962191621729F085
:1042D000E817F907D1F780E0089581E008959C017F
:1042E000FC0132969FEF80E04191461789F09F3F95
:1042F00019F4411101C0982F8F5F8630A9F79F3FB5
:1043000039F0F901E90FF11D97FDFA9562830895DF
:1043100008959C012A5F3F4FFC014281461301C072
:104320001282019682179307B9F708950C946F21B2
:104330000C948921029626E0FC0111922A95E9F756
:10434000089508950C94A12183E08093B9020C9400
:10435000A221811102C081E001C082E08093B902F4
:104360000C94A2210C94A92181E08093B9020C94B1
:10437000A2210C94B42108950C94BB210C94BC216F
:104380000C94BB210C94BB210C94BB21CF930E94B5
:10439000C2210E94A1170E94C021C0E08C2F0E9460
:1043A0008516892B29F4CF5FC530C1F780E001C0A5
:1043B00081E0CF91089508951F920F920FB60F924A
:1043C00011248F939F93AF93BF938091BA02811171
:1043D00013C08091E1029091E202A091E302B091BA
:1043E000E4024196A11DB11D8093E1029093E20287
:1043F000A093E302B093E402BF91AF919F918F919C
:104400000F900FBE0F901F9018958091E902843095
:1044100031F10E94DF071092BA0220E488E190E0B7
:104420000FB6F894A895809360000FBE20936000AB
:1044300083B7817F846083BF83B7816083BF7894B3
:10444000889583B78E7F83BF0FB6F894A895809127
:104450006000886180936000109260000FBE089534
:104460000E94800C0C94E30782E084BD93E095BD2C
:104470009AEF97BD80936E0008952FB7F8948091BE
:10448000E1029091E202A091E302B091E4022FBF19
:1044900008952FB7F8946091E1027091E202809143
:1044A000E3029091E4022FBF08959C014FB7F89466
:1044B0008091E1029091E202A091E302B091E402C6
:1044C0004FBF821B930B089578941F920F920FB6E3
:1044D0000F9211248F939F93AF93BF938091E1022A
:1044E0009091E202A091E302B091E4020196A11D35
:1044F000B11D8093E1029093E202A093E302B09396
:10450000E402BF91AF919F918F910F900FBE0F90DA
:104510001F90189581E08093E00080E28093D8009E
:104520001092C9008FE19EE40197F1F700C00000EE
:1045300087E090EBDC018093F2029093F302A0936A
:10454000F402B093F5029CE088E10FB6F894A895C8
:10455000809360000FBE90936000FFCF8091C902EE
:104560000895089522E02093E9002FEF3091E800AC
:10457000215035FD06C035ED3A95F1F700002111C7
:10458000F5CF2091E80025FF0BC040E050E066E049
:1045900070E00E949A258091E8008E778093E80071
:1045A0000895CF93DF9321E02093E9002FEF30911E
:1045B000E800215035FD06C035ED3A95F1F70000D1
:1045C0002111F5CF2091E80025FF14C0EC0140E057
:1045D00050E068E070E00E949A258091E8008E77B4
:1045E0008093E80088E0FE01A1ECB2E001900D921A
:1045F0008A95E1F7DF91CF9108958093BD02709382
:10460000BF026093BE028091E902843001F582E02E
:104610008093E9008FEF9091E800815095FD06C0EE
:1046200095ED9A95F1F700008111F5CF8091E800A2
:1046300085FF0DC040E050E063E070E08DEB92E05C
:104640000E949A258091E8008E778093E800089573
:10465000BC0184E00C94FD22BC0183E00C94FD229B
:1046600084EA9AE00E9466068091E802811109C0FE
:104670000E942B270E9488278091E200846080930B
:10468000E200089580EA9AE00E9466061092E8022D
:1046900008958CE99AE00E9466060C94B92188E995
:1046A0009AE00E9466066091E50281E0611101C016
:1046B00080E00C94A42184E99AE00E94660690911F
:1046C000E90281E0943009F080E06091E5020C9409
:1046D000A9212091BC022F5F822F62E30E94372A1A
:1046E000992319F02093BC0208951092BC02809186
:1046F000C002882371F18091E902843041F58091F4
:10470000E9008F702091EC00922F917020FD90E8CD
:10471000892B93E09093E9009091EB0090FF14C0F7
:104720009091EE0097FF10C09091E80095FF03C0B4
:104730001092F100F9CF9091E80090FF05C09091A0
:10474000E8009E779093E8008F708093E9001092C4
:10475000C002089542E061EC81E00E94A42642E29A
:1047600061EC82E00E94A42642E261EC83E00E94B8
:10477000A4269091E90281E0943009F080E06091F4
:10478000E5020C94B2218091EB02833009F461C000
:1047900030F4813071F0823009F49AC008958A3083
:1047A00009F486C08B3009F46CC0893009F0A8C0C8
:1047B00020C08091EA02813A09F0A2C08091E8000D
:1047C000877F8093E8008091EE029091EF02892B21
:1047D00021F468E081EC92E003C060E080E090E0CA
:1047E00070E00E94E5258091E8008B778093E800D7
:1047F00008958091EA02813209F082C08091EE0230
:104800009091EF02029708F07BC08091E800877FCB
:104810008093E8008091E80082FD05C08091E90264
:104820008111F8CF6DC02091F3008091F20090E0EB
:10483000922B029731F48091F100813011F0863093
:1048400021F48091F1008093C9028091E8008B7778
:1048500053C08091EA02813A09F052C08091EE0281
:104860009091EF02892B09F04BC08091E800877F7F
:104870008093E8008091E80080FFFCCF80911801D0
:1048800036C08091EA028132D9F58091EE02909192
:10489000EF02892BA9F58091E800877F8093E800DB
:1048A0000E94D9268091EC02809318010C94800C10
:1048B0008091EA02813221F58091E800877F809320
:1048C000E8000E94D9268091ED028093CA020895E3
:1048D0008091EA02813AA1F48091E800877F809379
:1048E000E8008091E80080FFFCCF8091CA028093AD
:1048F000F1008091E8008E778093E8000C94D9262F
:1049000008959FB7F8941092C0029FBF9091E9025A
:10491000943009F057C09091E9009F703091EC00FD
:10492000232F217030FD20E8922B23E02093E90013
:104930002091EB0020FF43C02091EE0027FF3FC0F5
:104940002091BB02222321F02091E80025FF37C0EF
:104950001092BB0226E03091E80035FD15C0309181
:10496000E902343061F53091EB0035FD28C021506B
:1049700021F481E08093BB0222C0EFE9FFE0319790
:10498000F1F700C00000E7CF8093F1008091E800CC
:1049900085FD0AC08091E80080FFFCCF8091E8008F
:1049A0008E778093E80006C08FB7F89421E02093BB
:1049B000C0028FBF9F709093E90080E008959F70C0
:1049C0009093E9008FEF089584B7877F84BF0FB677
:1049D000F894A8958091600088618093600010929F
:1049E00060000FBE90E080E80FB6F89480936100FD
:1049F000909361000FBE0C94B4210E942B270E945B
:104A00008827E2EEF0E080818460808378940C94C3
:104A10001C2A8CE091E00C94C0208091E902853042
:104A2000C9F480E99AE00E9466068091E902853027
:104A300079F40E9405228091E7028823B1F30E9455
:104A4000C621882391F30E9484250E94800CEDCF1B
:104A50000C943022089508950C942E25292F332785
:104A600023303105C9F060F42130310581F0223066
:104A7000310509F041C08BE590E026EF3AE040C0F7
:104A800021323105E1F02232310531F135C082E1C8
:104A900090E021E53BE034C099278130910549F051
:104AA00028F0029749F5E8EAFAE005C0E2EFFAE0FB
:104AB00002C0E6ECFAE0849190E09F0121C06330EF
:104AC0007105D0F4660F771FFB01EB50FE4F20817C
:104AD000318189E090E014C06330710568F4FB0116
:104AE000EE0FFF1FE151FE4F20813181FB01E451A8
:104AF000FE4F808190E004C080E090E020E030E054
:104B0000FA0131832083089580E189BD82E189BD66
:104B100009B400FEFDCF8091D8008F7D8093D8002E
:104B20008091E00082608093E0008091E00081FD50
:104B3000FCCF0895CF92DF92EF92FF920F931F93D5
:104B4000CF93DF93EC018B017A010E94F82681114B
:104B500033C0E114F10439F0F70180819181081B21
:104B6000190BC80FD91FC12CD12C0115110519F132
:104B70008091E80085FD16C08091E8008E778093D3
:104B8000E800E114F10449F0F70180819181C80E39
:104B9000D91ED182C08285E00FC00E94F8268823EA
:104BA00021F30AC089918093F10001501109FFEFB0
:104BB000CF1ADF0ADACF80E0DF91CF911F910F91FA
:104BC000FF90EF90DF90CF9008952091F002309108
:104BD000F1022617370748F06115710539F4209165
:104BE000E8002E772093E80001C0B901FC0120E025
:104BF0006115710579F18091E9028823F1F1853021
:104C0000F1F18091E80083FD3CC08091E80082FDD5
:104C10002EC08091E80080FFEBCF2091F3008091BF
:104C2000F20090E0922B6115710551F088309105EA
:104C300038F421912093F100615071090196F3CF6E
:104C400021E0089709F020E08091E8008E778093BA
:104C5000E800CECF2111CFCF0AC08091E90288238E
:104C600061F0853061F08091E80083FD0AC0809199
:104C7000E80082FFF2CF80E0089582E0089583E0AB
:104C8000089581E008952091F0023091F1022617F5
:104C9000370748F06115710539F42091E8002E7747
:104CA0002093E80001C0B901FC0120E06115710505
:104CB00091F18091E902882309F440C0853009F41C
:104CC0003FC08091E80083FD3DC08091E80082FDF7
:104CD0002FC08091E80080FFE9CF2091F300809100
:104CE000F20090E0922B6115710559F08830910522
:104CF00040F424912093F10031966150710901969E
:104D0000F2CF21E0089709F020E08091E8008E774B
:104D10008093E800CBCF2111CCCF0AC08091E9026B
:104D2000882361F0853061F08091E80083FD0AC03E
:104D30008091E80082FFF2CF80E0089582E008953C
:104D400083E0089581E00895982F973068F5909357
:104D5000E900981739F07091EC002091ED00509126
:104D6000F00003C0242F762F50E021FD02C09F5F8A
:104D7000ECCF3091EB003E7F3093EB003091ED00B3
:104D80003D7F3093ED003091EB0031603093EB00CC
:104D90007093EC002093ED005093F0002091EE0012
:104DA00027FDE5CF80E008958F708093E90081E0D2
:104DB00008958091EA0287FF11C08091E80082FD8A
:104DC00005C08091E9028111F8CF11C08091E800FF
:104DD0008B770BC08091E902882349F08091E8002D
:104DE00080FFF8CF8091E8008E778093E8000895E7
:104DF0002091E4003091E50095E64091EC00842F8D
:104E0000817040FF23C08091E80080FD1DC080912B
:104E1000E902882399F0853099F08091EB0085FDB7
:104E200011C04091E4005091E5002417350729F3A3
:104E3000915011F09A01E1CF84E0089582E0089545
:104E400083E0089581E0089580E008954091E800AE
:104E500042FFDDCF08950E9499270E94A127E0EE2E
:104E6000F0E0808181608083E8EDF0E080818F77E1
:104E7000808319BCA7EDB0E08C918E7F8C938081EC
:104E80008F7E80831092E80208950F931F93CF9333
:104E9000DF930E9499270E94A127C8EDD0E0888166
:104EA0008F77888388818068888388818F7D8883D5
:104EB00019BC1092E9021092E5021092E7021092DA
:104EC000E60200EE10E0F80180818B7F808388810C
:104ED0008160888342E060E080E00E94A426E1EEE9
:104EE000F0E080818E7F8083E2EEF0E0808181605F
:104EF0008083808188608083F80180818E7F8083B9
:104F0000888180618883DF91CF911F910F910895EF
:104F1000E8EDF0E080818F7E8083E7EDF0E0808136
:104F20008160808384E082BF81E08093E8020C94FA
:104F30004527E8EDF0E080818E7F80831092E200CB
:104F400008951092DA001092E10008951F920F92D6
:104F50000FB60F9211242F933F934F935F936F934C
:104F60007F938F939F93AF93BF93EF93FF93809122
:104F7000E10082FF0BC08091E20082FF07C08091B8
:104F8000E1008B7F8093E1000E9469238091DA0029
:104F900080FF1FC08091D80080FF1BC08091DA0085
:104FA0008E7F8093DA008091D90080FF0DC080E170
:104FB00089BD82E189BD09B400FEFDCF81E0809307
:104FC000E9020E94302305C019BC1092E9020E9438
:104FD00042238091E10080FF19C08091E20080FFB0
:104FE00015C08091E2008E7F8093E2008091E20004
:104FF00080618093E2008091D80080628093D80025
:1050000019BC85E08093E9020E944F238091E10062
:1050100084FF30C08091E20084FF2CC080E189BD14
:1050200082E189BD09B400FEFDCF8091D8008F7D5B
:105030008093D8008091E1008F7E8093E100809181
:10504000E2008F7E8093E2008091E2008160809395
:10505000E2008091E502882311F084E007C080918E
:10506000E30087FD02C081E001C083E08093E90294
:105070000E945B238091E10083FF29C08091E200C0
:1050800083FF25C08091E100877F8093E10082E06B
:105090008093E9021092E5028091E1008E7F809377
:1050A000E1008091E2008E7F8093E2008091E20037
:1050B00080618093E20042E060E080E00E94A426EC
:1050C0008091F00088608093F0000E944923FF9156
:1050D000EF91BF91AF919F918F917F916F915F9170
:1050E0004F913F912F910F900FBE0F901F901895E9
:1050F0001F920F920FB60F9211242F933F934F934D
:105100005F936F937F938F939F93AF93BF93CF934F
:10511000DF93EF93FF93C091E900CF708091EC0093
:10512000D82FD17080FDD0E81092E9008091F00076
:10513000877F8093F00078940E94BC281092E90049
:105140008091F00088608093F000CD2BCF70C093E9
:10515000E900FF91EF91DF91CF91BF91AF919F91C6
:105160008F917F916F915F914F913F912F910F9010
:105170000FBE0F901F9018951F93CF93DF93CDB75D
:10518000DEB7AA970FB6F894DEBF0FBECDBFEAEE2A
:10519000F2E08091F100819322E0E23FF207C9F74B
:1051A0000E94C3238091E80083FF2EC18091EA0210
:1051B0009091EB02492F50E04A30510508F024C18C
:1051C000FA01EE59FF4F0C94572A803821F08238AB
:1051D00009F01AC108C08091E6029091E702992374
:1051E00089F082600FC08091EE028F70873008F0E6
:1051F0000BC18093E9008091EB0085FB882780F943
:105200001092E9009091E800977F9093E8008093D6
:10521000F1001092F100D1C0282F2D7F09F0F4C0C9
:10522000882319F0823061F0EFC08091EC02813068
:1052300009F0EAC0933009F080E08093E7022EC0C5
:105240008091EC0281112AC08091EE028F702FEFC5
:10525000280F263008F0D8C08093E9002091EB0099
:1052600020FF1CC0933021F48091EB00806214C0B9
:105270009091EB0090619093EB0021E030E0A90168
:1052800002C0440F551F8A95E2F74093EA0010923E
:10529000EA008091EB0088608093EB001092E900B7
:1052A0008091E800877F8093E8000E94D926ACC0F7
:1052B0008111AAC01091EC021F778091E3008078E1
:1052C000812B8093E3008091E800877F8093E80042
:1052D0000E94D9268091E80080FFFCCF8091E300F6
:1052E00080688093E300111102C082E001C083E076
:1052F0008093E90289C08058823008F085C080918F
:10530000EC029091ED028C3D53E0950779F583E036
:105310008A838AE289834FB7F894DE01139620E0EE
:105320003EE051E2E32FF0E050935700E49120FF7C
:1053300003C0E295EF703F5FEF708E2F90E0EA3090
:1053400010F0C79601C0C0968D939D932F5F2431B6
:1053500049F74FBF8091E800877F8093E8006AE2B9
:1053600070E0CE0101960E94E52516C06091EE0224
:105370007091EF02AE014F5F5F4F0E942C25BC0180
:10538000892B09F441C09091E800977F9093E80041
:1053900089819A810E9443268091E8008B778093CF
:1053A000E80032C0803881F58091E800877F8093E3
:1053B000E8008091E5028093F1008091E8008E770B
:1053C00072CF811121C08091EC029091ED0299275A
:1053D0000297D4F48091E800877F8093E800809161
:1053E000EC028093E5020E94D9268091E5028111AA
:1053F00006C08091E30087FD02C081E001C084E027
:105400008093E9020E94AA238091E80083FF0AC0EA
:105410008091E800877F8093E8008091EB008062B4
:105420008093EB00AA960FB6F894DEBF0FBECDBFF7
:10543000DF91CF911F910895CF938091E902882346
:10544000A1F0C091E900CF709091EC00892F81709C
:1054500090FD80E8C82B1092E9008091E80083FD60
:105460000E94BC28CF70C093E900CF910895991B8A
:1054700079E004C0991F961708F0961B881F7A954B
:10548000C9F78095089597FB072E16F4009407D06E
:1054900077FD09D00E945D2A07FC05D03EF4909567
:1054A00081959F4F0895709561957F4F0895EE0FF8
:1054B000FF1F0590F491E02D0994AA1BBB1B51E13D
:1054C00007C0AA1FBB1FA617B70710F0A61BB70B74
:1054D000881F991F5A95A9F780959095BC01CD0119
:1054E0000895FB01DC0104C08D910190801921F425
:1054F00041505040C8F7881B990B0895F999FECF89
:1055000092BD81BDF89A992780B50895A8E1B0E0D1
:1055100042E050E00C94B22A262FF999FECF92BDBA
:1055200081BDF89A019700B4021639F01FBA20BD68
:105530000FB6F894FA9AF99A0FBE08950396272F9A
:105540000E948D2A0E948C2A252F0E948D2A242FAA
:105550000C948D2A0196272F0E948D2A0C948C2A58
:10556000DC01CB01FC01F999FECF06C0F2BDE1BD23
:10557000F89A319600B40D9241505040B8F7089512
:04558000F894FFCFCD
:10558400C8007C02280850011E0A1401AE22D12250
:10559400B2222C232823B12201E200E900EA00B55B
:1055A40000B600B700CD008301CC008A01920194BB
:1055B400012102230224022502260227022A02B321
:1055C40000B4006F007000818283E200E900EA0009
:1055D400B500B600B700CD008301CC008A0192016A
:1055E40094012102230224022502260227022A0210
:1055F400B300B4006F007000818283F0F1F4F5F61B
:10560400F767663696949392919030C69534353FF9
:105614003F3F006D6B5F64656C6179006D6B5F6922
:105624006E74657276616C006D6B5F6D61785F732B
:1056340070656564006D6B5F74696D655F746F5F41
:105644006D6178006D6B5F776865656C5F6D61781F
:105654005F7370656564006D6B5F776865656C5F2B
:1056640074696D655F746F5F6D617800407B2200C3
:0C5674000C850B630B080B210B3A0B009C
:00000001FF
